 cansdk

 Timestamp is 4da2a533 (Mon Apr 11 18:52:35 2011)

 Preferred load address is 10000000

 Start         Length     Name                   Class
 0001:00000000 00000004H .CRT$XCA                CODE
 0001:00000004 00000004H .CRT$XCZ                CODE
 0001:00000008 00000004H .CRT$XIA                CODE
 0001:0000000c 00000004H .CRT$XIZ                CODE
 0001:00000010 00000004H .CRT$XPA                CODE
 0001:00000014 00000004H .CRT$XPZ                CODE
 0001:00000018 00000004H .CRT$XTA                CODE
 0001:0000001c 00000004H .CRT$XTZ                CODE
 0001:00000020 00000428H .rdata                  CODE
 0001:00000448 00000023H .rdata$debug            CODE
 0001:0000046c 000010d0H .text                   CODE
 0001:0000153c 00000014H .idata$2                CODE
 0001:00001550 00000014H .idata$3                CODE
 0001:00001564 00000034H .idata$4                CODE
 0001:00001598 0000000cH .idata$6                CODE
 0001:000015b0 0000010bH .edata                  CODE
 0002:00000000 00000034H .idata$5                DATA
 0002:00000038 0000044cH .data                   DATA
 0002:00000484 0000000cH .bss                    DATA
 0003:00000000 000000b8H .pdata                  DATA

  Address         Publics by Value              Rva+Base       Lib:Object

 0000:00000000       ___safe_se_handler_count   00000000     <absolute>
 0000:00000000       ___safe_se_handler_table   00000000     <absolute>
 0001:00000000       __xc_a                     10001000     corelib0:crt0init.obj
 0001:00000004       __xc_z                     10001004     corelib0:crt0init.obj
 0001:00000008       __xi_a                     10001008     corelib0:crt0init.obj
 0001:0000000c       __xi_z                     1000100c     corelib0:crt0init.obj
 0001:00000010       __xp_a                     10001010     corelib0:crt0init.obj
 0001:00000014       __xp_z                     10001014     corelib0:crt0init.obj
 0001:00000018       __xt_a                     10001018     corelib0:crt0init.obj
 0001:0000001c       __xt_z                     1000101c     corelib0:crt0init.obj
 0001:0000003c       ??_C@_1O@IKMMPJPA@?$AA?9?$AA?9?$AA?$CF?$AAs?$AA?$AN?$AA?6?$AA?$AA@ 1000103c     cansdk_common_topaz_v1:cansdk.obj
 0001:0000004c       ??_C@_1DM@GMHGFAIO@?$AA?$CF?$AAs?$AA?3?$AA?5?$AA?5?$AAC?$AAr?$AAe?$AAa?$AAt?$AAe?$AAF?$AAi?$AAl?$AAe?$AA?5?$AAC?$AAA?$AAN?$AA?5?$AAf?$AAa?$AAi?$AAl?$AAe?$AAd?$AA?$CB?$AA?$AN?$AA?6?$AA?$AA@ 1000104c     cansdk_common_topaz_v1:cansdk.obj
 0001:00000088       ??_C@_1O@JNDDBHKG@?$AA?$CL?$AA?$CL?$AA?$CF?$AAs?$AA?$AN?$AA?6?$AA?$AA@ 10001088     cansdk_common_topaz_v1:cansdk.obj
 0001:00000098       ??_C@_1BM@JNLHLEII@?$AAC?$AAA?$AAN?$AAO?$AAp?$AAe?$AAn?$AAH?$AAa?$AAn?$AAd?$AAl?$AAe?$AA?$AA@ 10001098     cansdk_common_topaz_v1:cansdk.obj
 0001:000000b4       ??_C@_1DE@BBBAGJCD@?$AA?$CF?$AAs?$AA?3?$AA?5?$AAC?$AAl?$AAo?$AAs?$AAe?$AAH?$AAa?$AAn?$AAd?$AAl?$AAe?$AA?5?$AAf?$AAa?$AAi?$AAl?$AAe?$AAd?$AA?$CB?$AA?$AN?$AA?6?$AA?$AA@ 100010b4     cansdk_common_topaz_v1:cansdk.obj
 0001:000000e8       ??_C@_1BO@KCLGGKEE@?$AAC?$AAA?$AAN?$AAC?$AAl?$AAo?$AAs?$AAe?$AAH?$AAa?$AAn?$AAd?$AAl?$AAe?$AA?$AA@ 100010e8     cansdk_common_topaz_v1:cansdk.obj
 0001:00000108       ??_C@_1EO@HINKOHCP@?$AA?$CF?$AAs?$AA?3?$AA?5?$AAC?$AAA?$AAN?$AA_?$AAI?$AAO?$AAC?$AAT?$AAL?$AA_?$AAG?$AAE?$AAT?$AA_?$AAC?$AAL?$AAO?$AAC?$AAK?$AA_?$AAR?$AAA?$AAT?$AAE?$AA?5?$AAf?$AAa?$AAi@ 10001108     cansdk_common_topaz_v1:cansdk.obj
 0001:00000158       ??_C@_1CA@MCKKEMGA@?$AAC?$AAA?$AAN?$AAG?$AAe?$AAt?$AAC?$AAl?$AAo?$AAc?$AAk?$AAR?$AAa?$AAt?$AAe?$AA?$AA@ 10001158     cansdk_common_topaz_v1:cansdk.obj
 0001:00000178       ??_C@_1EO@CLKBDIHF@?$AA?$CF?$AAs?$AA?3?$AA?5?$AAC?$AAA?$AAN?$AA_?$AAI?$AAO?$AAC?$AAT?$AAL?$AA_?$AAS?$AAE?$AAT?$AA_?$AAC?$AAL?$AAO?$AAC?$AAK?$AA_?$AAR?$AAA?$AAT?$AAE?$AA?5?$AAf?$AAa?$AAi@ 10001178     cansdk_common_topaz_v1:cansdk.obj
 0001:000001c8       ??_C@_1CA@ECGMIBMG@?$AAC?$AAA?$AAN?$AAS?$AAe?$AAt?$AAC?$AAl?$AAo?$AAc?$AAk?$AAR?$AAa?$AAt?$AAe?$AA?$AA@ 100011c8     cansdk_common_topaz_v1:cansdk.obj
 0001:000001e8       ??_C@_1EC@CLBDPBLD@?$AA?$CF?$AAs?$AA?3?$AA?5?$AAC?$AAA?$AAN?$AA_?$AAI?$AAO?$AAC?$AAT?$AAL?$AA_?$AAT?$AAR?$AAA?$AAN?$AAS?$AAF?$AAE?$AAR?$AA?5?$AAf?$AAa?$AAi?$AAl?$AAe?$AAd?$AA?$CB?$AA?$AN?$AA?6@ 100011e8     cansdk_common_topaz_v1:cansdk.obj
 0001:0000022c       ??_C@_1BI@FGJOBHCA@?$AAC?$AAA?$AAN?$AAT?$AAr?$AAa?$AAn?$AAs?$AAf?$AAe?$AAr?$AA?$AA@ 1000122c     cansdk_common_topaz_v1:cansdk.obj
 0001:00000244       ??_C@_1DM@NBKLJOJK@?$AA?$CF?$AAs?$AA?3?$AA?5?$AAC?$AAA?$AAN?$AA_?$AAI?$AAO?$AAC?$AAT?$AAL?$AA_?$AAR?$AAE?$AAS?$AAE?$AAT?$AA?5?$AAf?$AAa?$AAi?$AAl?$AAe?$AAd?$AA?$CB?$AA?$AN?$AA?6?$AA?$AA@ 10001244     cansdk_common_topaz_v1:cansdk.obj
 0001:00000280       ??_C@_1BC@LLOOGMFM@?$AAC?$AAA?$AAN?$AAR?$AAe?$AAs?$AAe?$AAt?$AA?$AA@ 10001280     cansdk_common_topaz_v1:cansdk.obj
 0001:00000298       ??_C@_1EK@OEBDJKOD@?$AA?$CF?$AAs?$AA?3?$AA?5?$AAC?$AAA?$AAN?$AA_?$AAI?$AAO?$AAC?$AAT?$AAL?$AA_?$AAE?$AAN?$AAA?$AAB?$AAL?$AAE?$AA_?$AAS?$AAL?$AAA?$AAV?$AAE?$AA?5?$AAf?$AAa?$AAi?$AAl?$AAe@ 10001298     cansdk_common_topaz_v1:cansdk.obj
 0001:000002e4       ??_C@_1CA@OOMLPNPA@?$AAC?$AAA?$AAN?$AAE?$AAn?$AAa?$AAb?$AAl?$AAe?$AAT?$AAL?$AAP?$AAR?$AAI?$AAO?$AA?$AA@ 100012e4     cansdk_common_topaz_v1:cansdk.obj
 0001:00000308       ??_C@_1EM@CGHDBHII@?$AA?$CF?$AAs?$AA?3?$AA?5?$AAC?$AAA?$AAN?$AA_?$AAI?$AAO?$AAC?$AAT?$AAL?$AA_?$AAD?$AAI?$AAS?$AAA?$AAB?$AAL?$AAE?$AA_?$AAS?$AAL?$AAA?$AAV?$AAE?$AA?5?$AAf?$AAa?$AAi?$AAl@ 10001308     cansdk_common_topaz_v1:cansdk.obj
 0001:00000354       ??_C@_1CC@EDJGEKHH@?$AAC?$AAA?$AAN?$AAD?$AAi?$AAs?$AAa?$AAb?$AAl?$AAe?$AAT?$AAL?$AAP?$AAR?$AAI?$AAO?$AA?$AA@ 10001354     cansdk_common_topaz_v1:cansdk.obj
 0001:00000378       ??_C@_1BG@GEGOGKAC@?$AAC?$AAA?$AAN?$AAS?$AAe?$AAt?$AAM?$AAo?$AAd?$AAe?$AA?$AA@ 10001378     cansdk_common_topaz_v1:cansdk.obj
 0001:00000390       ??_C@_1FM@FOECPJNE@?$AA?$CK?$AA?$CK?$AA?$CK?$AA?$CK?$AA?$CK?$AA?5?$AAD?$AAL?$AAL?$AA?5?$AAP?$AAR?$AAO?$AAC?$AAE?$AAS?$AAS?$AA?5?$AAD?$AAE?$AAT?$AAA?$AAC?$AAH?$AA?5?$AAF?$AAR?$AAO?$AAM?$AA?5?$AAC?$AAA@ 10001390     cansdk_common_topaz_v1:cansdk.obj
 0001:000003f0       ??_C@_1FI@EPIKGHAK@?$AA?$CK?$AA?$CK?$AA?$CK?$AA?$CK?$AA?$CK?$AA?5?$AAD?$AAL?$AAL?$AA?5?$AAP?$AAR?$AAO?$AAC?$AAE?$AAS?$AAS?$AA?5?$AAA?$AAT?$AAT?$AAA?$AAC?$AAH?$AA?5?$AAT?$AAO?$AA?5?$AAC?$AAA?$AAN?$AA?5@ 100013f0     cansdk_common_topaz_v1:cansdk.obj
 0001:0000046c       CANOpenHandle              1000146c f   cansdk_common_topaz_v1:cansdk.obj
 0001:00000584       CANCloseHandle             10001584 f   cansdk_common_topaz_v1:cansdk.obj
 0001:0000067c       CANGetClockRate            1000167c f   cansdk_common_topaz_v1:cansdk.obj
 0001:00000798       CANSetClockRate            10001798 f   cansdk_common_topaz_v1:cansdk.obj
 0001:000008b4       CANTransfer                100018b4 f   cansdk_common_topaz_v1:cansdk.obj
 0001:000009d0       CANReset                   100019d0 f   cansdk_common_topaz_v1:cansdk.obj
 0001:00000aec       CANEnableTLPRIO            10001aec f   cansdk_common_topaz_v1:cansdk.obj
 0001:00000c08       CANDisableTLPRIO           10001c08 f   cansdk_common_topaz_v1:cansdk.obj
 0001:00000d24       CANSetMode                 10001d24 f   cansdk_common_topaz_v1:cansdk.obj
 0001:00000e54       DllEntry                   10001e54 f   cansdk_common_topaz_v1:cansdk.obj
 0001:00000f18       CreateFileW                10001f18 f   coredll:COREDLL.dll
 0001:00000f28       NKDbgPrintfW               10001f28 f   coredll:COREDLL.dll
 0001:00000f38       CloseHandle                10001f38 f   coredll:COREDLL.dll
 0001:00000f48       DeviceIoControl            10001f48 f   coredll:COREDLL.dll
 0001:00000f58       DisableThreadLibraryCalls  10001f58 f   coredll:COREDLL.dll
 0001:00000f68       RegisterDbgZones           10001f68 f   coredll:COREDLL.dll
 0001:00000f78       _DllEntryCRTStartup        10001f78 f   corelib0:pegdentry.obj
 0001:00000fe4       exit                       10001fe4 f   corelib0:cexit.obj
 0001:00001108       _exit                      10002108 f   corelib0:cexit.obj
 0001:00001128       _cexit                     10002128 f   corelib0:cexit.obj
 0001:00001140       _c_exit                    10002140 f   corelib0:cexit.obj
 0001:00001158       _initterm                  10002158 f   corelib0:crt0dat.obj
 0001:000011a4       _cinit                     100021a4 f   corelib0:crt0dat.obj
 0001:000011d4       __security_init_cookie     100021d4 f   corelib0:seccinit.obj
 0001:0000126c       __crt_ExitProcess          1000226c f   corelib0:exitproc_proxy.obj
 0001:00001298       GetCurrentProcess          10002298 f i corelib0:exitproc_proxy.obj
 0001:000012b0       _onexit                    100022b0 f   corelib0:onexit.obj
 0001:0000148c       atexit                     1000248c f   corelib0:onexit.obj
 0001:000014dc       free                       100024dc f   corelib1:COREDLL.dll
 0001:000014ec       __security_gen_cookie2     100024ec f   corelib1:COREDLL.dll
 0001:000014fc       realloc                    100024fc f   corelib1:COREDLL.dll
 0001:0000150c       malloc                     1000250c f   corelib1:COREDLL.dll
 0001:0000151c       _msize                     1000251c f   corelib1:COREDLL.dll
 0001:0000152c       TerminateProcess           1000252c f   coredll:COREDLL.dll
 0001:0000153c       __IMPORT_DESCRIPTOR_COREDLL 1000253c     coredll:COREDLL.dll
 0001:00001550       __NULL_IMPORT_DESCRIPTOR   10002550     coredll:COREDLL.dll
 0002:00000000       __imp_CreateFileW          10003000     coredll:COREDLL.dll
 0002:00000004       __imp_NKDbgPrintfW         10003004     coredll:COREDLL.dll
 0002:00000008       __imp_CloseHandle          10003008     coredll:COREDLL.dll
 0002:0000000c       __imp_DeviceIoControl      1000300c     coredll:COREDLL.dll
 0002:00000010       __imp_DisableThreadLibraryCalls 10003010     coredll:COREDLL.dll
 0002:00000014       __imp_RegisterDbgZones     10003014     coredll:COREDLL.dll
 0002:00000018       __imp_free                 10003018     corelib1:COREDLL.dll
 0002:0000001c       __imp___security_gen_cookie2 1000301c     corelib1:COREDLL.dll
 0002:00000020       __imp_realloc              10003020     corelib1:COREDLL.dll
 0002:00000024       __imp_malloc               10003024     corelib1:COREDLL.dll
 0002:00000028       __imp__msize               10003028     corelib1:COREDLL.dll
 0002:0000002c       __imp_TerminateProcess     1000302c     coredll:COREDLL.dll
 0002:00000030       \177COREDLL_NULL_THUNK_DATA 10003030     coredll:COREDLL.dll
 0002:00000038       dpCurSettings              10003038     cansdk_common_topaz_v1:cansdk.obj
 0002:0000047c       __security_cookie          1000347c     corelib0:seccinit.obj
 0002:00000480       __security_cookie_complement 10003480     corelib0:seccinit.obj
 0002:00000484       _exitflag                  10003484     corelib0:cexit.obj
 0002:00000488       __onexitend                10003488     <common>
 0002:0000048c       __onexitbegin              1000348c     <common>

 entry point at        0001:00000f78

 Static symbols

 0001:00001004       doexit                     10002004 f   corelib0:cexit.obj
